LX51 LINKER/LOCATER V3.58                                                               02/22/2012  09:49:47  PAGE 1


LX51 LINKER/LOCATER V3.58, INVOKED BY:
D:\KEIL\C51\BIN\LX51.EXE STARTUP.obj, Main.obj TO nRF24LE1 CLASSES (XDATA (X:0X0-X:0X3FF, X:0XFA00-X:0XFFFF), HDATA (X:0
>> X0-X:0X3FF, X:0XFA00-X:0XFFFF), CODE (C:0X0-C:0X3FFF), CONST (C:0X0-C:0X3FFF), ECODE (C:0X0-C:0X3FFF), HCONST (C:0X0-
>> C:0X3FFF))


CPU MODE:     8051 MODE
MEMORY MODEL: COMPACT


INPUT MODULES INCLUDED:
  STARTUP.obj (?C_STARTUP)
         COMMENT TYPE 0: AX51 V2.09
  Main.obj (MAIN)
         COMMENT TYPE 0: C51 V7.06
  D:\KEIL\C51\LIB\C51C.LIB (?C_INIT)
         COMMENT TYPE 1: A51 / ASM51 Assembler
  D:\KEIL\C51\LIB\C51C.LIB (?C?CLDPTR)
         COMMENT TYPE 1: A51 / ASM51 Assembler
  D:\KEIL\C51\LIB\C51C.LIB (?C?CSTOPTR)
         COMMENT TYPE 1: A51 / ASM51 Assembler
  D:\KEIL\C51\LIB\C51C.LIB (?C?ULCMP)
         COMMENT TYPE 1: A51 / ASM51 Assembler
  D:\KEIL\C51\LIB\C51C.LIB (?C?LSTPDATA)
         COMMENT TYPE 1: A51 / ASM51 Assembler
  D:\KEIL\C51\LIB\C51C.LIB (?C?LSTKPDATA)
         COMMENT TYPE 1: A51 / ASM51 Assembler


ACTIVE MEMORY CLASSES OF MODULE:  nRF24LE1 (?C_STARTUP)

BASE        START       END         USED      MEMORY CLASS
==========================================================
X:000000H   X:000000H   X:0003FFH             XDATA
            X:00FA00H   X:00FFFFH               
X:000000H   X:000000H   X:0003FFH             HDATA
            X:00FA00H   X:00FFFFH               
C:000000H   C:000000H   C:003FFFH   0004A8H   CODE
C:000000H   C:000000H   C:003FFFH             CONST
C:000000H   C:000000H   C:003FFFH             ECODE
B00:0000H   C:000000H   C:003FFFH             HCONST
I:000000H   I:000000H   I:0000FFH   000001H   IDATA
X:000000H   X:000000H   X:0000FFH   000015H   PDATA
I:000000H   I:000000H   I:00007FH   00001DH   DATA


MEMORY MAP OF MODULE:  nRF24LE1 (?C_STARTUP)


START     STOP      LENGTH    ALIGN  RELOC    MEMORY CLASS   SEGMENT NAME
=========================================================================

* * * * * * * * * * *   D A T A   M E M O R Y   * * * * * * * * * * * * *
000000H   000007H   000008H   ---    AT..     DATA           "REG BANK 0"
000008H   00001BH   000014H   BYTE   UNIT     DATA           ?DT?MAIN
00001CH   00001FH   000004H   ---    ---      **GAP**
000020H   000020H   000001H   BYTE   BITADDR  DATA           ?BA?MAIN
000021H   000021H   000001H   BYTE   UNIT     IDATA          ?STACK

* * * * * * * * * * *   C O D E   M E M O R Y   * * * * * * * * * * * * *
000000H   000002H   000003H   ---    OFFS..   CODE           ?CO?STARTUP?3
000003H   00000AH   000008H   BYTE   UNIT     CODE           ?PR?ADC_START?MAIN
00000BH   00000DH   000003H   BYTE   OFFS..   CODE           ?MAIN?0000B
00000EH   000049H   00003CH   BYTE   UNIT     CODE           ?PR?TX_MODE?MAIN
00004AH   00004AH   000001H   ---    ---      **GAP**
00004BH   00004DH   000003H   BYTE   OFFS..   CODE           ?MAIN?0004B
LX51 LINKER/LOCATER V3.58                                                             02/22/2012  09:49:47  PAGE 2


00004EH   000067H   00001AH   BYTE   UNIT     CODE           ?PR?IO_INIT?MAIN
000068H   00006AH   000003H   BYTE   UNIT     CODE           ?PR?RTC2_IRQ?MAIN
00006BH   00006DH   000003H   BYTE   OFFS..   CODE           ?MAIN?0006B
00006EH   0001BBH   00014EH   BYTE   UNIT     CODE           ?PR?MAIN?MAIN
0001BCH   000247H   00008CH   BYTE   UNIT     CODE           ?C_C51STARTUP
000248H   0002B8H   000071H   BYTE   UNIT     CODE           ?C?LIB_CODE
0002B9H   000310H   000058H   BYTE   UNIT     CODE           ?PR?RF_IRQ?MAIN
000311H   000366H   000056H   BYTE   UNIT     CODE           ?PR?RF_INIT?MAIN
000367H   0003A6H   000040H   BYTE   UNIT     CODE           ?PR?_DELAY?MAIN
0003A7H   0003D8H   000032H   BYTE   UNIT     CODE           ?PR?_SPI_READ_BUF?MAIN
0003D9H   00040AH   000032H   BYTE   UNIT     CODE           ?PR?_SPI_WRITE_BUF?MAIN
00040BH   00041EH   000014H   BYTE   UNIT     CODE           ?PR?_SPI_RW?MAIN
00041FH   000432H   000014H   BYTE   UNIT     CODE           ?C_INITSEG
000433H   000443H   000011H   BYTE   UNIT     CODE           ?PR?_SPI_RW_REG?MAIN
000444H   000452H   00000FH   BYTE   UNIT     CODE           ?PR?RTC2_INIT?MAIN
000453H   00045FH   00000DH   BYTE   UNIT     CODE           ?PR?_SPI_READ?MAIN
000460H   00046CH   00000DH   BYTE   UNIT     CODE           ?PR?RTC0_INIT?MAIN
00046DH   000479H   00000DH   BYTE   UNIT     CODE           ?PR?RTC0_IRQ?MAIN
00047AH   000485H   00000CH   BYTE   UNIT     CODE           ?PR?RX_MODE?MAIN
000486H   00048FH   00000AH   BYTE   UNIT     CODE           ?PR?ADC_INIT?MAIN
000490H   000498H   000009H   BYTE   UNIT     CODE           ?PR?PD_MODE?MAIN
000499H   0004A0H   000008H   BYTE   UNIT     CODE           ?PR?GET_ADC_VALUE?MAIN
0004A1H   0004A4H   000004H   BYTE   UNIT     CODE           ?PR?RTC2_ON?MAIN
0004A5H   0004A8H   000004H   BYTE   UNIT     CODE           ?PR?RTC2_OFF?MAIN

* * * * * * * * * * *  X D A T A   M E M O R Y  * * * * * * * * * * * * *
000000H   00000FH   000010H   BYTE   INPAGE   PDATA          _PDATA_GROUP_
000010H   000014H   000005H   BYTE   INPAGE   PDATA          ?PD?MAIN



OVERLAY MAP OF MODULE:   nRF24LE1 (?C_STARTUP)


FUNCTION/MODULE             PDATA_GROUP
--> CALLED FUNCTION/MODULE  START  STOP
=======================================
?C_C51STARTUP               ----- -----
  +--> ?PR?MAIN?MAIN
  +--> ?C_INITSEG

MAIN/MAIN                   0000H 0005H
  +--> ?PR?IO_INIT?MAIN
  +--> ?PR?RF_INIT?MAIN
  +--> ?PR?_DELAY?MAIN
  +--> ?PR?RX_MODE?MAIN
  +--> ?PR?PD_MODE?MAIN
  +--> ?PR?TX_MODE?MAIN

IO_INIT/MAIN                ----- -----
  +--> ?PR?_DELAY?MAIN

_DELAY/MAIN                 0006H 0007H

RF_INIT/MAIN                ----- -----
  +--> ?PR?_DELAY?MAIN
  +--> ?PR?_SPI_WRITE_BUF?MAIN
  +--> ?PR?_SPI_RW_REG?MAIN

_SPI_WRITE_BUF/MAIN         0006H 000AH
  +--> ?PR?_SPI_RW?MAIN

_SPI_RW/MAIN                ----- -----

_SPI_RW_REG/MAIN            ----- -----
LX51 LINKER/LOCATER V3.58                                                             02/22/2012  09:49:47  PAGE 3


  +--> ?PR?_SPI_RW?MAIN

RX_MODE/MAIN                ----- -----
  +--> ?PR?_SPI_RW_REG?MAIN

PD_MODE/MAIN                ----- -----
  +--> ?PR?_SPI_RW_REG?MAIN

TX_MODE/MAIN                ----- -----
  +--> ?PR?_SPI_RW_REG?MAIN
  +--> ?PR?_SPI_WRITE_BUF?MAIN
  +--> ?PR?_DELAY?MAIN

?C_INITSEG                  ----- -----

*** NEW ROOT **************

RF_IRQ/MAIN                 ----- -----
  +--> ?PR?_SPI_READ?MAIN
  +--> ?PR?_SPI_READ_BUF?MAIN
  +--> ?PR?_SPI_RW_REG?MAIN

_SPI_READ/MAIN              ----- -----
  +--> ?PR?_SPI_RW?MAIN

_SPI_READ_BUF/MAIN          000BH 000FH
  +--> ?PR?_SPI_RW?MAIN

*** NEW ROOT **************

RTC2_IRQ/MAIN               ----- -----

*** NEW ROOT **************

RTC0_IRQ/MAIN               ----- -----



PUBLIC SYMBOLS OF MODULE:  nRF24LE1 (?C_STARTUP)


      VALUE       CLASS    TYPE      PUBLIC SYMBOL NAME
      =================================================
      0200000BH   PDATA    BYTE      ?_SPI_Read_Buf?BYTE
      02000006H   PDATA    BYTE      ?_SPI_Write_Buf?BYTE
      01000248H   CODE     ---       ?C?CLDPTR
      00000000H   NUMBER   ---       ?C?CODESEG
      01000261H   CODE     ---       ?C?CSTOPTR
      010002A0H   CODE     ---       ?C?LSTKPDATA
      01000294H   CODE     ---       ?C?LSTPDATA
      01000283H   CODE     ---       ?C?ULCMP
      00000000H   NUMBER   ---       ?C?XDATASEG
      01000203H   CODE     ---       ?C_START
      01000000H   CODE     NEAR LAB  ?C_STARTUP
      0100037BH   CODE     ---       _delay
      01000453H   CODE     ---       _SPI_Read
      010003A7H   CODE     ---       _SPI_Read_Buf
      01000415H   CODE     ---       _SPI_RW
      01000433H   CODE     ---       _SPI_RW_Reg
      010003D9H   CODE     ---       _SPI_Write_Buf
*SFR* 000000D0H.6 DATA     BIT       AC
*SFR* 000000E0H   DATA     BYTE      ACC
      01000486H   CODE     ---       adc_init
      01000003H   CODE     ---       adc_start
*SFR* 000000D3H   DATA     BYTE      ADCCON1
LX51 LINKER/LOCATER V3.58                                                             02/22/2012  09:49:47  PAGE 4


*SFR* 000000D2H   DATA     BYTE      ADCCON2
*SFR* 000000D1H   DATA     BYTE      ADCCON3
*SFR* 000000D4H   DATA     BYTE      ADCDATH
*SFR* 000000D5H   DATA     BYTE      ADCDATL
*SFR* 000000D8H   DATA     BYTE      ADCON
*SFR* 000000EFH   DATA     BYTE      ARCON
*SFR* 000000F0H   DATA     BYTE      B
*SFR* 000000D8H.7 DATA     BIT       BD
*SFR* 000000C2H   DATA     WORD      CC1
*SFR* 000000C4H   DATA     WORD      CC2
*SFR* 000000C6H   DATA     WORD      CC3
*SFR* 000000C1H   DATA     BYTE      CCEN
*SFR* 000000C3H   DATA     BYTE      CCH1
*SFR* 000000C5H   DATA     BYTE      CCH2
*SFR* 000000C7H   DATA     BYTE      CCH3
*SFR* 000000C2H   DATA     BYTE      CCL1
*SFR* 000000C4H   DATA     BYTE      CCL2
*SFR* 000000C6H   DATA     BYTE      CCL3
*SFR* 000000DDH   DATA     BYTE      CCPDATIA
*SFR* 000000DEH   DATA     BYTE      CCPDATIB
*SFR* 000000DFH   DATA     BYTE      CCPDATO
*SFR* 000000A3H   DATA     BYTE      CLKCTRL
*SFR* 000000ADH   DATA     BYTE      CLKLFCTRL
*SFR* 000000DBH   DATA     BYTE      COMPCON
*SFR* 000000CAH   DATA     WORD      CRC
*SFR* 000000CBH   DATA     BYTE      CRCH
*SFR* 000000CAH   DATA     BYTE      CRCL
*SFR* 000000D0H.7 DATA     BIT       CY
*SFR* 00000083H   DATA     BYTE      DPH
*SFR* 00000085H   DATA     BYTE      DPH1
*SFR* 00000082H   DATA     BYTE      DPL
*SFR* 00000084H   DATA     BYTE      DPL1
*SFR* 00000092H   DATA     BYTE      DPS
*SFR* 000000A8H.7 DATA     BIT       EA
*SFR* 000000A8H.4 DATA     BIT       ES0
*SFR* 000000A8H.1 DATA     BIT       ET0
*SFR* 000000A8H.3 DATA     BIT       ET1
*SFR* 000000A8H.5 DATA     BIT       ET2
*SFR* 000000A8H   DATA     BIT       EX0
*SFR* 000000A8H.2 DATA     BIT       EX1
*SFR* 000000B8H.7 DATA     BIT       EXEN2
*SFR* 000000C0H.7 DATA     BIT       EXF2
*SFR* 000000D0H.5 DATA     BIT       F0
*SFR* 000000FAH   DATA     BYTE      FCR
*SFR* 000000FBH   DATA     BYTE      FDCR
*SFR* 000000F9H   DATA     BYTE      FPCR
*SFR* 000000F8H   DATA     BYTE      FSR
      01000499H   CODE     ---       get_adc_value
*SFR* 000000C8H.5 DATA     BIT       I2FR
*SFR* 000000C8H.6 DATA     BIT       I3FR
      00000012H   DATA     ---       id_buf
*SFR* 00000088H.1 DATA     BIT       IE0
*SFR* 00000088H.3 DATA     BIT       IE1
*SFR* 000000A8H   DATA     BYTE      IEN0
*SFR* 000000B8H   DATA     BYTE      IEN1
*SFR* 000000F8H.3 DATA     BIT       INFEN
*SFR* 000000A6H   DATA     BYTE      INTEXP
      0100004EH   CODE     ---       io_init
*SFR* 000000A9H   DATA     BYTE      IP0
*SFR* 000000B9H   DATA     BYTE      IP1
*SFR* 000000C0H   DATA     BYTE      IRCON
*SFR* 00000088H   DATA     BIT       IT0
*SFR* 00000088H.2 DATA     BIT       IT1
*SFR* 00000080H   DATA     BIT       LED0
*SFR* 00000080H.1 DATA     BIT       LED1
LX51 LINKER/LOCATER V3.58                                                             02/22/2012  09:49:47  PAGE 5


*SFR* 00000080H.2 DATA     BIT       LED2
*SFR* 00000080H.3 DATA     BIT       LED3
*SFR* 00000080H.4 DATA     BIT       LED4
*SFR* 00000080H.5 DATA     BIT       LED5
*SFR* 00000080H.6 DATA     BIT       LED6
*SFR* 00000090H.2 DATA     BIT       LED7
*SFR* 00000090H.3 DATA     BIT       LED8
*SFR* 00000090H.4 DATA     BIT       LED9
      0100006EH   CODE     ---       main
      00000020H.4 DATA     BIT       MAX_RT
*SFR* 000000F8H.7 DATA     BIT       MCDIS
*SFR* 000000E9H   DATA     BYTE      MD0
*SFR* 000000EAH   DATA     BYTE      MD1
*SFR* 000000EBH   DATA     BYTE      MD2
*SFR* 000000ECH   DATA     BYTE      MD3
*SFR* 000000EDH   DATA     BYTE      MD4
*SFR* 000000EEH   DATA     BYTE      MD5
*SFR* 000000A7H   DATA     BYTE      MEMCON
*SFR* 000000B8H.4 DATA     BIT       MISC
*SFR* 000000C0H.4 DATA     BIT       MISCF
*SFR* 000000C9H   DATA     BYTE      MPAGE
*SFR* 000000AEH   DATA     BYTE      OPMCON
*SFR* 000000D0H.2 DATA     BIT       OV
*SFR* 000000D0H   DATA     BIT       P
*SFR* 00000080H   DATA     BYTE      P0
*SFR* 00000080H   DATA     BIT       P00
*SFR* 00000080H.1 DATA     BIT       P01
*SFR* 00000080H.2 DATA     BIT       P02
*SFR* 00000080H.3 DATA     BIT       P03
*SFR* 00000080H.4 DATA     BIT       P04
*SFR* 00000080H.5 DATA     BIT       P05
*SFR* 00000080H.6 DATA     BIT       P06
*SFR* 00000080H.7 DATA     BIT       P07
*SFR* 0000009EH   DATA     BYTE      P0CON
*SFR* 00000093H   DATA     BYTE      P0DIR
*SFR* 00000090H   DATA     BYTE      P1
*SFR* 00000090H   DATA     BIT       P10
*SFR* 00000090H.1 DATA     BIT       P11
*SFR* 00000090H.2 DATA     BIT       P12
*SFR* 00000090H.3 DATA     BIT       P13
*SFR* 00000090H.4 DATA     BIT       P14
*SFR* 00000090H.5 DATA     BIT       P15
*SFR* 00000090H.6 DATA     BIT       P16
*SFR* 00000090H.7 DATA     BIT       P17
*SFR* 0000009FH   DATA     BYTE      P1CON
*SFR* 00000094H   DATA     BYTE      P1DIR
*SFR* 000000A0H   DATA     BYTE      P2
*SFR* 000000A0H   DATA     BIT       P20
*SFR* 000000A0H.1 DATA     BIT       P21
*SFR* 000000A0H.2 DATA     BIT       P22
*SFR* 000000A0H.3 DATA     BIT       P23
*SFR* 000000A0H.4 DATA     BIT       P24
*SFR* 000000A0H.5 DATA     BIT       P25
*SFR* 000000A0H.6 DATA     BIT       P26
*SFR* 000000A0H.7 DATA     BIT       P27
*SFR* 00000097H   DATA     BYTE      P2CON
*SFR* 00000095H   DATA     BYTE      P2DIR
*SFR* 000000B0H   DATA     BYTE      P3
*SFR* 000000B0H   DATA     BIT       P30
*SFR* 000000B0H.1 DATA     BIT       P31
*SFR* 000000B0H.2 DATA     BIT       P32
*SFR* 000000B0H.3 DATA     BIT       P33
*SFR* 000000B0H.4 DATA     BIT       P34
*SFR* 000000B0H.5 DATA     BIT       P35
*SFR* 000000B0H.6 DATA     BIT       P36
LX51 LINKER/LOCATER V3.58                                                             02/22/2012  09:49:47  PAGE 6


*SFR* 000000B0H.7 DATA     BIT       P37
*SFR* 0000008FH   DATA     BYTE      P3CON
*SFR* 00000096H   DATA     BYTE      P3DIR
*SFR* 00000087H   DATA     BYTE      PCON
      01000490H   CODE     ---       PD_Mode
*SFR* 000000DCH   DATA     BYTE      POFCON
*SFR* 000000A0H   DATA     BYTE      PPAGE_SFR
*SFR* 000000D0H   DATA     BYTE      PSW
*SFR* 000000B2H   DATA     BYTE      PWMCON
*SFR* 000000A1H   DATA     BYTE      PWMDC0
*SFR* 000000A2H   DATA     BYTE      PWMDC1
*SFR* 000000A4H   DATA     BYTE      PWRDWN
*SFR* 00000098H.2 DATA     BIT       RB80
*SFR* 000000F8H.1 DATA     BIT       RDEND
*SFR* 000000F8H.2 DATA     BIT       RDIS
*SFR* 000000F8H.4 DATA     BIT       RDYN
*SFR* 00000098H.4 DATA     BIT       REN0
*SFR* 000000B8H.1 DATA     BIT       RF
      01000311H   CODE     ---       rf_init
      010002B9H   CODE     ---       RF_IRQ
*SFR* 000000E8H   DATA     BIT       RFCE
*SFR* 000000E8H.2 DATA     BIT       RFCKEN
*SFR* 000000E8H   DATA     BYTE      RFCON
*SFR* 000000E8H.1 DATA     BIT       RFCSN
*SFR* 000000C0H.1 DATA     BIT       RFF
*SFR* 000000B8H   DATA     BIT       RFSPI
*SFR* 000000C0H   DATA     BIT       RFSPIF
*SFR* 00000098H   DATA     BIT       RI0
*SFR* 000000D6H   DATA     BYTE      RNGCTL
*SFR* 000000D7H   DATA     BYTE      RNGDAT
*SFR* 000000D0H.3 DATA     BIT       RS0
*SFR* 000000D0H.4 DATA     BIT       RS1
*SFR* 000000B1H   DATA     BYTE      RSTREAS
      01000460H   CODE     ---       rtc0_init
      0100046DH   CODE     ---       RTC0_IRQ
      01000444H   CODE     ---       rtc2_init
      01000068H   CODE     ---       RTC2_IRQ
      010004A5H   CODE     ---       rtc2_off
      010004A1H   CODE     ---       rtc2_on
*SFR* 000000B4H   DATA     BYTE      RTC2CMP0
*SFR* 000000B5H   DATA     BYTE      RTC2CMP1
*SFR* 000000B3H   DATA     BYTE      RTC2CON
*SFR* 000000B6H   DATA     BYTE      RTC2CPT00
*SFR* 000000ABH   DATA     BYTE      RTC2CPT01
*SFR* 000000ACH   DATA     BYTE      RTC2CPT10
      00000008H   DATA     ---       rx_buf
      00000020H.6 DATA     BIT       RX_DR
      0100047AH   CODE     ---       RX_Mode
*SFR* 00000099H   DATA     BYTE      S0BUF
*SFR* 00000098H   DATA     BYTE      S0CON
*SFR* 000000BAH   DATA     BYTE      S0RELH
*SFR* 000000AAH   DATA     BYTE      S0RELL
*SFR* 00000090H.5 DATA     BIT       S1
*SFR* 00000090H.6 DATA     BIT       S2
*SFR* 00000090H.4 DATA     BIT       S3
*SFR* 00000098H.7 DATA     BIT       SM0
*SFR* 00000098H.6 DATA     BIT       SM1
*SFR* 00000098H.5 DATA     BIT       SM20
*SFR* 00000081H   DATA     BYTE      SP
*SFR* 000000B8H.2 DATA     BIT       SPI
*SFR* 000000C0H.2 DATA     BIT       SPIF
*SFR* 000000FCH   DATA     BYTE      SPIMCON0
*SFR* 000000FDH   DATA     BYTE      SPIMCON1
*SFR* 000000FFH   DATA     BYTE      SPIMDAT
*SFR* 000000FEH   DATA     BYTE      SPIMSTAT
LX51 LINKER/LOCATER V3.58                                                             02/22/2012  09:49:47  PAGE 7


*SFR* 000000E4H   DATA     BYTE      SPIRCON0
*SFR* 000000E5H   DATA     BYTE      SPIRCON1
*SFR* 000000E7H   DATA     BYTE      SPIRDAT
*SFR* 000000E6H   DATA     BYTE      SPIRSTAT
*SFR* 000000BCH   DATA     BYTE      SPISCON0
*SFR* 000000BDH   DATA     BYTE      SPISCON1
*SFR* 000000BFH   DATA     BYTE      SPISDAT
*SFR* 000000B7H   DATA     BYTE      SPISRDSZ
*SFR* 000000BEH   DATA     BYTE      SPISSTAT
      00000020H   DATA     BYTE      sta
*SFR* 000000F8H.6 DATA     BIT       STP
*SFR* 000000CCH   DATA     WORD      T2
*SFR* 000000C8H.2 DATA     BIT       T2CM
*SFR* 000000C8H   DATA     BYTE      T2CON
*SFR* 000000C8H   DATA     BIT       T2I0
*SFR* 000000C8H.1 DATA     BIT       T2I1
*SFR* 000000C8H.7 DATA     BIT       T2PS
*SFR* 000000C8H.3 DATA     BIT       T2R0
*SFR* 000000C8H.4 DATA     BIT       T2R1
*SFR* 00000098H.3 DATA     BIT       TB80
*SFR* 00000088H   DATA     BYTE      TCON
*SFR* 00000088H.5 DATA     BIT       TF0
*SFR* 00000088H.7 DATA     BIT       TF1
*SFR* 000000C0H.6 DATA     BIT       TF2
*SFR* 0000008CH   DATA     BYTE      TH0
*SFR* 0000008DH   DATA     BYTE      TH1
*SFR* 000000CDH   DATA     BYTE      TH2
*SFR* 00000098H.1 DATA     BIT       TI0
*SFR* 0000008AH   DATA     BYTE      TL0
*SFR* 0000008BH   DATA     BYTE      TL1
*SFR* 000000CCH   DATA     BYTE      TL2
*SFR* 00000089H   DATA     BYTE      TMOD
*SFR* 00000088H.4 DATA     BIT       TR0
*SFR* 00000088H.6 DATA     BIT       TR1
      02000010H   PDATA    ---       TX_ADDRESS
      00000020H.5 DATA     BIT       TX_DS
      0100000EH   CODE     ---       TX_Mode
*SFR* 000000E2H   DATA     BYTE      W2CON0
*SFR* 000000E1H   DATA     BYTE      W2CON1
*SFR* 000000DAH   DATA     BYTE      W2DAT
*SFR* 000000D9H   DATA     BYTE      W2SADR
*SFR* 000000AFH   DATA     BYTE      WDSV
*SFR* 000000F8H.5 DATA     BIT       WEN
*SFR* 000000F8H   DATA     BIT       WPEN
*SFR* 000000A5H   DATA     BYTE      WUCON
*SFR* 000000C0H.5 DATA     BIT       WUF
*SFR* 000000B8H.5 DATA     BIT       WUIRQ
*SFR* 000000CFH   DATA     BYTE      WUOPC0
*SFR* 000000CEH   DATA     BYTE      WUOPC1
*SFR* 000000B8H.3 DATA     BIT       WUPIN
*SFR* 000000C0H.3 DATA     BIT       WUPINF



SYMBOL TABLE OF MODULE:  nRF24LE1 (?C_STARTUP)

      VALUE       REP       CLASS    TYPE      SYMBOL NAME
      ====================================================
      ---         MODULE    ---      ---       ?C_STARTUP
      01000000H   PUBLIC    CODE     NEAR LAB  ?C_STARTUP
      000000E0H   SFRSYM    DATA     BYTE      ACC
      000000F0H   SFRSYM    DATA     BYTE      B
      00000083H   SFRSYM    DATA     BYTE      DPH
      00000082H   SFRSYM    DATA     BYTE      DPL
      000000A0H   SFRSYM    DATA     BYTE      PPAGE_SFR
LX51 LINKER/LOCATER V3.58                                                             02/22/2012  09:49:47  PAGE 8


      00000081H   SFRSYM    DATA     BYTE      SP
      00000000H   SYMBOL    NUMBER   ---       IBPSTACK
      00000100H   SYMBOL    NUMBER   ---       IBPSTACKTOP
      00000080H   SYMBOL    NUMBER   ---       IDATALEN
      010001BFH   SYMBOL    CODE     NEAR LAB  IDATALOOP
      00000000H   SYMBOL    NUMBER   ---       PBPSTACK
      00010000H   SYMBOL    NUMBER   ---       PBPSTACKTOP
      00000000H   SYMBOL    NUMBER   ---       PDATALEN
      00000000H   SYMBOL    NUMBER   ---       PDATASTART
      00000000H   SYMBOL    NUMBER   ---       PPAGE
      00000000H   SYMBOL    NUMBER   ---       PPAGEENABLE
      010001BCH   SYMBOL    CODE     NEAR LAB  STARTUP1
      00000000H   SYMBOL    NUMBER   ---       XBPSTACK
      00010000H   SYMBOL    NUMBER   ---       XBPSTACKTOP
      00000000H   SYMBOL    NUMBER   ---       XDATALEN
      00000000H   SYMBOL    NUMBER   ---       XDATASTART

      01000000H   BLOCK     CODE     NEAR LAB  LVL=0
      01000000H   LINE      CODE     ---       #92
      ---         BLOCKEND  ---      ---       LVL=0

      010001BCH   BLOCK     CODE     NEAR LAB  LVL=0
      010001BCH   LINE      CODE     ---       #99
      010001BEH   LINE      CODE     ---       #100
      010001BFH   LINE      CODE     ---       #101
      010001C0H   LINE      CODE     ---       #102
      010001C2H   LINE      CODE     ---       #151
      010001C5H   LINE      CODE     ---       #155
      ---         BLOCKEND  ---      ---       LVL=0

      ---         MODULE    ---      ---       MAIN
      00000020H.4 PUBLIC    DATA     BIT       MAX_RT
      00000012H   PUBLIC    DATA     ---       id_buf
      00000020H.5 PUBLIC    DATA     BIT       TX_DS
      00000020H.6 PUBLIC    DATA     BIT       RX_DR
      00000020H   PUBLIC    DATA     BYTE      sta
      02000010H   PUBLIC    PDATA    ---       TX_ADDRESS
      00000008H   PUBLIC    DATA     ---       rx_buf
      0100006EH   PUBLIC    CODE     ---       main
      01000499H   PUBLIC    CODE     ---       get_adc_value
      01000003H   PUBLIC    CODE     ---       adc_start
      01000486H   PUBLIC    CODE     ---       adc_init
      0100004EH   PUBLIC    CODE     ---       io_init
      0100046DH   PUBLIC    CODE     ---       RTC0_IRQ
      01000068H   PUBLIC    CODE     ---       RTC2_IRQ
      010004A5H   PUBLIC    CODE     ---       rtc2_off
      010004A1H   PUBLIC    CODE     ---       rtc2_on
      01000460H   PUBLIC    CODE     ---       rtc0_init
      01000444H   PUBLIC    CODE     ---       rtc2_init
      010002B9H   PUBLIC    CODE     ---       RF_IRQ
      01000311H   PUBLIC    CODE     ---       rf_init
      0100047AH   PUBLIC    CODE     ---       RX_Mode
      0100000EH   PUBLIC    CODE     ---       TX_Mode
      01000490H   PUBLIC    CODE     ---       PD_Mode
      02000006H   PUBLIC    PDATA    BYTE      ?_SPI_Write_Buf?BYTE
      010003D9H   PUBLIC    CODE     ---       _SPI_Write_Buf
      0200000BH   PUBLIC    PDATA    BYTE      ?_SPI_Read_Buf?BYTE
      010003A7H   PUBLIC    CODE     ---       _SPI_Read_Buf
      01000453H   PUBLIC    CODE     ---       _SPI_Read
      01000433H   PUBLIC    CODE     ---       _SPI_RW_Reg
      01000415H   PUBLIC    CODE     ---       _SPI_RW
      0100037BH   PUBLIC    CODE     ---       _delay
      00000098H.3 SFRSYM    DATA     BIT       TB80
      000000BEH   SFRSYM    DATA     BYTE      SPISSTAT
      000000C8H   SFRSYM    DATA     BIT       T2I0
LX51 LINKER/LOCATER V3.58                                                             02/22/2012  09:49:47  PAGE 9


      000000C3H   SFRSYM    DATA     BYTE      CCH1
      00000080H   SFRSYM    DATA     BYTE      P0
      000000C8H.1 SFRSYM    DATA     BIT       T2I1
      000000DFH   SFRSYM    DATA     BYTE      CCPDATO
      000000C5H   SFRSYM    DATA     BYTE      CCH2
      00000090H   SFRSYM    DATA     BYTE      P1
      000000C7H   SFRSYM    DATA     BYTE      CCH3
      000000A0H   SFRSYM    DATA     BYTE      P2
      00000098H.5 SFRSYM    DATA     BIT       SM20
      000000B0H   SFRSYM    DATA     BYTE      P3
      00000090H.5 SFRSYM    DATA     BIT       S1
      000000D0H.6 SFRSYM    DATA     BIT       AC
      000000C2H   SFRSYM    DATA     BYTE      CCL1
      00000090H.6 SFRSYM    DATA     BIT       S2
      000000C4H   SFRSYM    DATA     BYTE      CCL2
      00000080H   SFRSYM    DATA     BIT       LED0
      00000090H.4 SFRSYM    DATA     BIT       S3
      000000D8H.7 SFRSYM    DATA     BIT       BD
      000000B8H   SFRSYM    DATA     BIT       RFSPI
      000000A8H.7 SFRSYM    DATA     BIT       EA
      000000CCH   SFRSYM    DATA     WORD      T2
      000000C6H   SFRSYM    DATA     BYTE      CCL3
      000000B7H   SFRSYM    DATA     BYTE      SPISRDSZ
      00000080H.1 SFRSYM    DATA     BIT       LED1
      00000080H.2 SFRSYM    DATA     BIT       LED2
      00000080H.3 SFRSYM    DATA     BIT       LED3
      000000C8H.3 SFRSYM    DATA     BIT       T2R0
      00000080H.4 SFRSYM    DATA     BIT       LED4
      000000C8H.4 SFRSYM    DATA     BIT       T2R1
      00000080H.5 SFRSYM    DATA     BIT       LED5
      00000080H.6 SFRSYM    DATA     BIT       LED6
      00000090H.2 SFRSYM    DATA     BIT       LED7
      000000A8H   SFRSYM    DATA     BYTE      IEN0
      00000090H.3 SFRSYM    DATA     BIT       LED8
      000000B8H   SFRSYM    DATA     BYTE      IEN1
      000000A5H   SFRSYM    DATA     BYTE      WUCON
      00000085H   SFRSYM    DATA     BYTE      DPH1
      00000090H.4 SFRSYM    DATA     BIT       LED9
      000000DBH   SFRSYM    DATA     BYTE      COMPCON
      000000A3H   SFRSYM    DATA     BYTE      CLKCTRL
      00000084H   SFRSYM    DATA     BYTE      DPL1
      000000C8H.5 SFRSYM    DATA     BIT       I2FR
      000000B8H.3 SFRSYM    DATA     BIT       WUPIN
      000000C8H.6 SFRSYM    DATA     BIT       I3FR
      000000FFH   SFRSYM    DATA     BYTE      SPIMDAT
      000000C0H.7 SFRSYM    DATA     BIT       EXF2
      00000098H.4 SFRSYM    DATA     BIT       REN0
      000000C8H.2 SFRSYM    DATA     BIT       T2CM
      000000B8H.1 SFRSYM    DATA     BIT       RF
      000000B8H.5 SFRSYM    DATA     BIT       WUIRQ
      000000E7H   SFRSYM    DATA     BYTE      SPIRDAT
      000000C1H   SFRSYM    DATA     BYTE      CCEN
      000000E2H   SFRSYM    DATA     BYTE      W2CON0
      000000BFH   SFRSYM    DATA     BYTE      SPISDAT
      000000D0H.7 SFRSYM    DATA     BIT       CY
      000000E1H   SFRSYM    DATA     BYTE      W2CON1
      000000FBH   SFRSYM    DATA     BYTE      FDCR
      000000E8H   SFRSYM    DATA     BIT       RFCE
      000000CBH   SFRSYM    DATA     BYTE      CRCH
      00000081H   SFRSYM    DATA     BYTE      SP
      000000D0H.2 SFRSYM    DATA     BIT       OV
      000000CAH   SFRSYM    DATA     BYTE      CRCL
      000000ADH   SFRSYM    DATA     BYTE      CLKLFCTRL
      000000B1H   SFRSYM    DATA     BYTE      RSTREAS
      000000C8H.7 SFRSYM    DATA     BIT       T2PS
LX51 LINKER/LOCATER V3.58                                                             02/22/2012  09:49:47  PAGE 10


      000000F9H   SFRSYM    DATA     BYTE      FPCR
      000000B8H.4 SFRSYM    DATA     BIT       MISC
      000000A1H   SFRSYM    DATA     BYTE      PWMDC0
      000000B4H   SFRSYM    DATA     BYTE      RTC2CMP0
      000000A2H   SFRSYM    DATA     BYTE      PWMDC1
      000000B5H   SFRSYM    DATA     BYTE      RTC2CMP1
      00000080H   SFRSYM    DATA     BIT       P00
      000000BAH   SFRSYM    DATA     BYTE      S0RELH
      00000090H   SFRSYM    DATA     BIT       P10
      00000080H.1 SFRSYM    DATA     BIT       P01
      00000087H   SFRSYM    DATA     BYTE      PCON
      000000A0H   SFRSYM    DATA     BIT       P20
      00000090H.1 SFRSYM    DATA     BIT       P11
      00000080H.2 SFRSYM    DATA     BIT       P02
      000000B0H   SFRSYM    DATA     BIT       P30
      000000A0H.1 SFRSYM    DATA     BIT       P21
      00000090H.2 SFRSYM    DATA     BIT       P12
      00000080H.3 SFRSYM    DATA     BIT       P03
      000000C0H.2 SFRSYM    DATA     BIT       SPIF
      000000F8H.2 SFRSYM    DATA     BIT       RDIS
      000000B0H.1 SFRSYM    DATA     BIT       P31
      000000A0H.2 SFRSYM    DATA     BIT       P22
      00000090H.3 SFRSYM    DATA     BIT       P13
      00000080H.4 SFRSYM    DATA     BIT       P04
      000000AAH   SFRSYM    DATA     BYTE      S0RELL
      000000B0H.2 SFRSYM    DATA     BIT       P32
      000000A0H.3 SFRSYM    DATA     BIT       P23
      00000090H.4 SFRSYM    DATA     BIT       P14
      00000080H.5 SFRSYM    DATA     BIT       P05
      000000D9H   SFRSYM    DATA     BYTE      W2SADR
      00000089H   SFRSYM    DATA     BYTE      TMOD
      00000088H   SFRSYM    DATA     BYTE      TCON
      000000B0H.3 SFRSYM    DATA     BIT       P33
      000000A0H.4 SFRSYM    DATA     BIT       P24
      00000090H.5 SFRSYM    DATA     BIT       P15
      00000080H.6 SFRSYM    DATA     BIT       P06
      000000B0H.4 SFRSYM    DATA     BIT       P34
      000000A0H.5 SFRSYM    DATA     BIT       P25
      00000090H.6 SFRSYM    DATA     BIT       P16
      00000080H.7 SFRSYM    DATA     BIT       P07
      000000C2H   SFRSYM    DATA     WORD      CC1
      000000B0H.5 SFRSYM    DATA     BIT       P35
      000000A0H.6 SFRSYM    DATA     BIT       P26
      00000090H.7 SFRSYM    DATA     BIT       P17
      000000C4H   SFRSYM    DATA     WORD      CC2
      000000B0H.6 SFRSYM    DATA     BIT       P36
      000000A0H.7 SFRSYM    DATA     BIT       P27
      000000C6H   SFRSYM    DATA     WORD      CC3
      000000B0H.7 SFRSYM    DATA     BIT       P37
      000000E8H.2 SFRSYM    DATA     BIT       RFCKEN
      000000F8H   SFRSYM    DATA     BIT       WPEN
      000000DDH   SFRSYM    DATA     BYTE      CCPDATIA
      000000DEH   SFRSYM    DATA     BYTE      CCPDATIB
      00000088H.1 SFRSYM    DATA     BIT       IE0
      000000F8H.4 SFRSYM    DATA     BIT       RDYN
      00000088H.3 SFRSYM    DATA     BIT       IE1
      000000CFH   SFRSYM    DATA     BYTE      WUOPC0
      000000F0H   SFRSYM    DATA     BYTE      B
      000000E9H   SFRSYM    DATA     BYTE      MD0
      000000CEH   SFRSYM    DATA     BYTE      WUOPC1
      000000A7H   SFRSYM    DATA     BYTE      MEMCON
      000000EAH   SFRSYM    DATA     BYTE      MD1
      000000D7H   SFRSYM    DATA     BYTE      RNGDAT
      000000EBH   SFRSYM    DATA     BYTE      MD2
      000000ECH   SFRSYM    DATA     BYTE      MD3
LX51 LINKER/LOCATER V3.58                                                             02/22/2012  09:49:47  PAGE 11


      000000EDH   SFRSYM    DATA     BYTE      MD4
      000000AFH   SFRSYM    DATA     BYTE      WDSV
      000000EEH   SFRSYM    DATA     BYTE      MD5
      000000E0H   SFRSYM    DATA     BYTE      ACC
      000000DCH   SFRSYM    DATA     BYTE      POFCON
      000000A8H.4 SFRSYM    DATA     BIT       ES0
      000000A8H.1 SFRSYM    DATA     BIT       ET0
      000000A9H   SFRSYM    DATA     BYTE      IP0
      000000A8H.3 SFRSYM    DATA     BIT       ET1
      00000088H.5 SFRSYM    DATA     BIT       TF0
      000000B9H   SFRSYM    DATA     BYTE      IP1
      000000A8H.5 SFRSYM    DATA     BIT       ET2
      00000098H   SFRSYM    DATA     BIT       RI0
      00000088H.7 SFRSYM    DATA     BIT       TF1
      000000C0H   SFRSYM    DATA     BIT       RFSPIF
      000000C0H.6 SFRSYM    DATA     BIT       TF2
      000000FCH   SFRSYM    DATA     BYTE      SPIMCON0
      000000D6H   SFRSYM    DATA     BYTE      RNGCTL
      0000008CH   SFRSYM    DATA     BYTE      TH0
      000000A8H   SFRSYM    DATA     BIT       EX0
      00000098H.1 SFRSYM    DATA     BIT       TI0
      00000088H   SFRSYM    DATA     BIT       IT0
      000000FDH   SFRSYM    DATA     BYTE      SPIMCON1
      0000008DH   SFRSYM    DATA     BYTE      TH1
      000000A8H.2 SFRSYM    DATA     BIT       EX1
      00000088H.2 SFRSYM    DATA     BIT       IT1
      000000CDH   SFRSYM    DATA     BYTE      TH2
      000000AEH   SFRSYM    DATA     BYTE      OPMCON
      000000D0H   SFRSYM    DATA     BIT       P
      00000098H.7 SFRSYM    DATA     BIT       SM0
      0000008AH   SFRSYM    DATA     BYTE      TL0
      00000098H.6 SFRSYM    DATA     BIT       SM1
      000000E4H   SFRSYM    DATA     BYTE      SPIRCON0
      0000008BH   SFRSYM    DATA     BYTE      TL1
      000000E5H   SFRSYM    DATA     BYTE      SPIRCON1
      000000CCH   SFRSYM    DATA     BYTE      TL2
      000000BCH   SFRSYM    DATA     BYTE      SPISCON0
      000000BDH   SFRSYM    DATA     BYTE      SPISCON1
      000000D0H.3 SFRSYM    DATA     BIT       RS0
      00000088H.4 SFRSYM    DATA     BIT       TR0
      000000D0H.4 SFRSYM    DATA     BIT       RS1
      000000B2H   SFRSYM    DATA     BYTE      PWMCON
      00000088H.6 SFRSYM    DATA     BIT       TR1
      000000CAH   SFRSYM    DATA     WORD      CRC
      000000A6H   SFRSYM    DATA     BYTE      INTEXP
      000000C0H.3 SFRSYM    DATA     BIT       WUPINF
      000000FAH   SFRSYM    DATA     BYTE      FCR
      000000D3H   SFRSYM    DATA     BYTE      ADCCON1
      000000D2H   SFRSYM    DATA     BYTE      ADCCON2
      00000083H   SFRSYM    DATA     BYTE      DPH
      000000D1H   SFRSYM    DATA     BYTE      ADCCON3
      000000C0H.1 SFRSYM    DATA     BIT       RFF
      00000093H   SFRSYM    DATA     BYTE      P0DIR
      00000082H   SFRSYM    DATA     BYTE      DPL
      0000009EH   SFRSYM    DATA     BYTE      P0CON
      00000099H   SFRSYM    DATA     BYTE      S0BUF
      00000094H   SFRSYM    DATA     BYTE      P1DIR
      0000009FH   SFRSYM    DATA     BYTE      P1CON
      00000095H   SFRSYM    DATA     BYTE      P2DIR
      000000B8H.7 SFRSYM    DATA     BIT       EXEN2
      000000DAH   SFRSYM    DATA     BYTE      W2DAT
      00000097H   SFRSYM    DATA     BYTE      P2CON
      00000096H   SFRSYM    DATA     BYTE      P3DIR
      000000A4H   SFRSYM    DATA     BYTE      PWRDWN
      00000098H   SFRSYM    DATA     BYTE      S0CON
LX51 LINKER/LOCATER V3.58                                                             02/22/2012  09:49:47  PAGE 12


      0000008FH   SFRSYM    DATA     BYTE      P3CON
      000000B6H   SFRSYM    DATA     BYTE      RTC2CPT00
      000000D8H   SFRSYM    DATA     BYTE      ADCON
      000000ACH   SFRSYM    DATA     BYTE      RTC2CPT10
      000000ABH   SFRSYM    DATA     BYTE      RTC2CPT01
      000000C8H   SFRSYM    DATA     BYTE      T2CON
      00000092H   SFRSYM    DATA     BYTE      DPS
      000000F8H.5 SFRSYM    DATA     BIT       WEN
      000000F8H   SFRSYM    DATA     BYTE      FSR
      000000D4H   SFRSYM    DATA     BYTE      ADCDATH
      000000C9H   SFRSYM    DATA     BYTE      MPAGE
      000000B8H.2 SFRSYM    DATA     BIT       SPI
      000000F8H.1 SFRSYM    DATA     BIT       RDEND
      000000D5H   SFRSYM    DATA     BYTE      ADCDATL
      000000F8H.3 SFRSYM    DATA     BIT       INFEN
      000000F8H.7 SFRSYM    DATA     BIT       MCDIS
      000000C0H.5 SFRSYM    DATA     BIT       WUF
      000000C0H.4 SFRSYM    DATA     BIT       MISCF
      000000EFH   SFRSYM    DATA     BYTE      ARCON
      000000D0H.5 SFRSYM    DATA     BIT       F0
      000000F8H.6 SFRSYM    DATA     BIT       STP
      000000FEH   SFRSYM    DATA     BYTE      SPIMSTAT
      000000E8H   SFRSYM    DATA     BYTE      RFCON
      000000D0H   SFRSYM    DATA     BYTE      PSW
      00000098H.2 SFRSYM    DATA     BIT       RB80
      000000C0H   SFRSYM    DATA     BYTE      IRCON
      000000E8H.1 SFRSYM    DATA     BIT       RFCSN
      000000E6H   SFRSYM    DATA     BYTE      SPIRSTAT
      000000B3H   SFRSYM    DATA     BYTE      RTC2CON

      01000367H   BLOCK     CODE     ---       LVL=0
      ---         BLOCKEND  ---      ---       LVL=0

      0100037BH   BLOCK     CODE     ---       LVL=0
      00000006H   SYMBOL    DATA     WORD      x
      00000004H   SYMBOL    DATA     WORD      i
      02000006H   SYMBOL    PDATA    WORD      j
      0100037BH   BLOCK     CODE     NEAR LAB  LVL=1
      00000004H   SYMBOL    DATA     WORD      i
      02000006H   SYMBOL    PDATA    WORD      j
      ---         BLOCKEND  ---      ---       LVL=1
      0100037BH   LINE      CODE     ---       #83
      0100037BH   LINE      CODE     ---       #84
      0100037BH   LINE      CODE     ---       #86
      0100037EH   LINE      CODE     ---       #87
      01000385H   LINE      CODE     ---       #88
      01000385H   LINE      CODE     ---       #89
      0100038DH   LINE      CODE     ---       #91
      0100039FH   LINE      CODE     ---       #92
      010003A6H   LINE      CODE     ---       #93
      ---         BLOCKEND  ---      ---       LVL=0

      0100040BH   BLOCK     CODE     ---       LVL=0
      ---         BLOCKEND  ---      ---       LVL=0

      01000415H   BLOCK     CODE     ---       LVL=0
      00000007H   SYMBOL    DATA     BYTE      value
      01000415H   LINE      CODE     ---       #97
      01000415H   LINE      CODE     ---       #98
      01000415H   LINE      CODE     ---       #99
      01000417H   LINE      CODE     ---       #101
      0100041CH   LINE      CODE     ---       #103
      0100041EH   LINE      CODE     ---       #104
      ---         BLOCKEND  ---      ---       LVL=0

LX51 LINKER/LOCATER V3.58                                                             02/22/2012  09:49:47  PAGE 13


      01000433H   BLOCK     CODE     ---       LVL=0
      00000007H   SYMBOL    DATA     BYTE      reg
      00000005H   SYMBOL    DATA     BYTE      value
      01000433H   BLOCK     CODE     NEAR LAB  LVL=1
      00000006H   SYMBOL    DATA     BYTE      status
      ---         BLOCKEND  ---      ---       LVL=1
      01000433H   LINE      CODE     ---       #108
      01000433H   LINE      CODE     ---       #109
      01000433H   LINE      CODE     ---       #112
      01000435H   LINE      CODE     ---       #113
      0100043AH   LINE      CODE     ---       #114
      0100043FH   LINE      CODE     ---       #115
      01000441H   LINE      CODE     ---       #117
      01000443H   LINE      CODE     ---       #118
      ---         BLOCKEND  ---      ---       LVL=0

      01000453H   BLOCK     CODE     ---       LVL=0
      00000007H   SYMBOL    DATA     BYTE      reg
      01000453H   BLOCK     CODE     NEAR LAB  LVL=1
      00000007H   SYMBOL    DATA     BYTE      reg_val
      ---         BLOCKEND  ---      ---       LVL=1
      01000453H   LINE      CODE     ---       #122
      01000453H   LINE      CODE     ---       #123
      01000453H   LINE      CODE     ---       #126
      01000455H   LINE      CODE     ---       #127
      01000458H   LINE      CODE     ---       #128
      0100045DH   LINE      CODE     ---       #129
      0100045FH   LINE      CODE     ---       #131
      0100045FH   LINE      CODE     ---       #132
      ---         BLOCKEND  ---      ---       LVL=0

      010003A7H   BLOCK     CODE     ---       LVL=0
      00000007H   SYMBOL    DATA     BYTE      reg
      0200000CH   SYMBOL    PDATA    ---       pBuf
      0200000FH   SYMBOL    PDATA    BYTE      bytes
      010003A9H   BLOCK     CODE     NEAR LAB  LVL=1
      00000006H   SYMBOL    DATA     BYTE      status
      00000005H   SYMBOL    DATA     BYTE      byte_ctr
      ---         BLOCKEND  ---      ---       LVL=1
      010003A7H   LINE      CODE     ---       #137
      010003A9H   LINE      CODE     ---       #138
      010003A9H   LINE      CODE     ---       #141
      010003A9H   LINE      CODE     ---       #142
      010003AEH   LINE      CODE     ---       #144
      010003B9H   LINE      CODE     ---       #145
      010003D4H   LINE      CODE     ---       #147
      010003D6H   LINE      CODE     ---       #149
      010003D8H   LINE      CODE     ---       #150
      ---         BLOCKEND  ---      ---       LVL=0

      010003D9H   BLOCK     CODE     ---       LVL=0
      00000007H   SYMBOL    DATA     BYTE      reg
      02000007H   SYMBOL    PDATA    ---       pBuf
      0200000AH   SYMBOL    PDATA    BYTE      bytes
      010003DBH   BLOCK     CODE     NEAR LAB  LVL=1
      00000006H   SYMBOL    DATA     BYTE      status
      00000005H   SYMBOL    DATA     BYTE      byte_ctr
      ---         BLOCKEND  ---      ---       LVL=1
      010003D9H   LINE      CODE     ---       #154
      010003DBH   LINE      CODE     ---       #155
      010003DBH   LINE      CODE     ---       #158
      010003DBH   LINE      CODE     ---       #159
      010003E0H   LINE      CODE     ---       #160
      010003EBH   LINE      CODE     ---       #161
      01000406H   LINE      CODE     ---       #162
LX51 LINKER/LOCATER V3.58                                                             02/22/2012  09:49:47  PAGE 14


      01000408H   LINE      CODE     ---       #163
      0100040AH   LINE      CODE     ---       #164
      ---         BLOCKEND  ---      ---       LVL=0

      01000490H   BLOCK     CODE     ---       LVL=0
      01000490H   LINE      CODE     ---       #168
      01000490H   LINE      CODE     ---       #169
      01000490H   LINE      CODE     ---       #170
      01000492H   LINE      CODE     ---       #171
      ---         BLOCKEND  ---      ---       LVL=0

      0100000EH   BLOCK     CODE     ---       LVL=0
      0100000EH   LINE      CODE     ---       #176
      0100000EH   LINE      CODE     ---       #177
      0100000EH   LINE      CODE     ---       #178
      01000010H   LINE      CODE     ---       #179
      01000017H   LINE      CODE     ---       #180
      0100001AH   LINE      CODE     ---       #181
      0100001DH   LINE      CODE     ---       #182
      01000020H   LINE      CODE     ---       #185
      01000023H   LINE      CODE     ---       #186
      01000026H   LINE      CODE     ---       #187
      01000029H   LINE      CODE     ---       #188
      0100002CH   LINE      CODE     ---       #189
      0100002FH   LINE      CODE     ---       #190
      0100003EH   LINE      CODE     ---       #191
      01000040H   LINE      CODE     ---       #192
      01000047H   LINE      CODE     ---       #193
      01000049H   LINE      CODE     ---       #194
      ---         BLOCKEND  ---      ---       LVL=0

      0100047AH   BLOCK     CODE     ---       LVL=0
      0100047AH   LINE      CODE     ---       #199
      0100047AH   LINE      CODE     ---       #200
      0100047AH   LINE      CODE     ---       #201
      0100047CH   LINE      CODE     ---       #202
      01000483H   LINE      CODE     ---       #203
      01000485H   LINE      CODE     ---       #204
      ---         BLOCKEND  ---      ---       LVL=0

      01000311H   BLOCK     CODE     ---       LVL=0
      01000311H   LINE      CODE     ---       #208
      01000311H   LINE      CODE     ---       #209
      01000311H   LINE      CODE     ---       #210
      01000313H   LINE      CODE     ---       #211
      01000315H   LINE      CODE     ---       #212
      01000317H   LINE      CODE     ---       #214
      0100031EH   LINE      CODE     ---       #216
      0100032EH   LINE      CODE     ---       #217
      0100033EH   LINE      CODE     ---       #219
      01000345H   LINE      CODE     ---       #220
      0100034BH   LINE      CODE     ---       #221
      01000352H   LINE      CODE     ---       #222
      01000359H   LINE      CODE     ---       #223
      01000360H   LINE      CODE     ---       #224
      ---         BLOCKEND  ---      ---       LVL=0

      010002B9H   BLOCK     CODE     ---       LVL=0
      010002B9H   LINE      CODE     ---       #229
      010002D2H   LINE      CODE     ---       #231
      010002D9H   LINE      CODE     ---       #232
      010002DCH   LINE      CODE     ---       #233
      010002DCH   LINE      CODE     ---       #234
      010002ECH   LINE      CODE     ---       #235
      010002F3H   LINE      CODE     ---       #236
LX51 LINKER/LOCATER V3.58                                                             02/22/2012  09:49:47  PAGE 15


      010002F3H   LINE      CODE     ---       #238
      010002FAH   LINE      CODE     ---       #239
      ---         BLOCKEND  ---      ---       LVL=0

      01000444H   BLOCK     CODE     ---       LVL=0
      01000444H   LINE      CODE     ---       #244
      01000444H   LINE      CODE     ---       #245
      01000444H   LINE      CODE     ---       #246
      01000447H   LINE      CODE     ---       #247
      0100044AH   LINE      CODE     ---       #248
      0100044DH   LINE      CODE     ---       #249
      01000450H   LINE      CODE     ---       #250
      01000452H   LINE      CODE     ---       #251
      ---         BLOCKEND  ---      ---       LVL=0

      01000460H   BLOCK     CODE     ---       LVL=0
      01000460H   LINE      CODE     ---       #256
      01000460H   LINE      CODE     ---       #257
      01000460H   LINE      CODE     ---       #258
      01000462H   LINE      CODE     ---       #259
      01000465H   LINE      CODE     ---       #260
      01000467H   LINE      CODE     ---       #261
      0100046AH   LINE      CODE     ---       #262
      0100046CH   LINE      CODE     ---       #265
      ---         BLOCKEND  ---      ---       LVL=0

      010004A1H   BLOCK     CODE     ---       LVL=0
      010004A1H   LINE      CODE     ---       #271
      010004A1H   LINE      CODE     ---       #272
      010004A1H   LINE      CODE     ---       #273
      010004A4H   LINE      CODE     ---       #274
      ---         BLOCKEND  ---      ---       LVL=0

      010004A5H   BLOCK     CODE     ---       LVL=0
      010004A5H   LINE      CODE     ---       #278
      010004A5H   LINE      CODE     ---       #279
      010004A5H   LINE      CODE     ---       #280
      010004A8H   LINE      CODE     ---       #281
      ---         BLOCKEND  ---      ---       LVL=0

      01000068H   BLOCK     CODE     ---       LVL=0
      01000068H   LINE      CODE     ---       #285
      01000068H   LINE      CODE     ---       #287
      0100006AH   LINE      CODE     ---       #288
      ---         BLOCKEND  ---      ---       LVL=0

      0100046DH   BLOCK     CODE     ---       LVL=0
      0100046DH   LINE      CODE     ---       #293
      0100046DH   LINE      CODE     ---       #296
      0100046FH   LINE      CODE     ---       #297
      01000472H   LINE      CODE     ---       #298
      01000475H   LINE      CODE     ---       #299
      01000477H   LINE      CODE     ---       #300
      01000479H   LINE      CODE     ---       #301
      ---         BLOCKEND  ---      ---       LVL=0

      0100004EH   BLOCK     CODE     ---       LVL=0
      0100004EH   LINE      CODE     ---       #305
      0100004EH   LINE      CODE     ---       #306
      0100004EH   LINE      CODE     ---       #307
      01000051H   LINE      CODE     ---       #308
      01000054H   LINE      CODE     ---       #310
      0100005AH   LINE      CODE     ---       #311
      01000061H   LINE      CODE     ---       #312
      01000067H   LINE      CODE     ---       #313
LX51 LINKER/LOCATER V3.58                                                             02/22/2012  09:49:47  PAGE 16


      ---         BLOCKEND  ---      ---       LVL=0

      01000486H   BLOCK     CODE     ---       LVL=0
      01000486H   LINE      CODE     ---       #317
      01000486H   LINE      CODE     ---       #318
      01000486H   LINE      CODE     ---       #319
      01000489H   LINE      CODE     ---       #320
      0100048CH   LINE      CODE     ---       #321
      0100048FH   LINE      CODE     ---       #322
      ---         BLOCKEND  ---      ---       LVL=0

      01000003H   BLOCK     CODE     ---       LVL=0
      01000003H   BLOCK     CODE     NEAR LAB  LVL=1
      00000007H   SYMBOL    DATA     BYTE      temp
      ---         BLOCKEND  ---      ---       LVL=1
      01000003H   LINE      CODE     ---       #327
      01000003H   LINE      CODE     ---       #328
      01000003H   LINE      CODE     ---       #330
      01000005H   LINE      CODE     ---       #331
      01000008H   LINE      CODE     ---       #332
      0100000AH   LINE      CODE     ---       #334
      ---         BLOCKEND  ---      ---       LVL=0

      01000499H   BLOCK     CODE     ---       LVL=0
      01000499H   BLOCK     CODE     NEAR LAB  LVL=1
      00000007H   SYMBOL    DATA     BYTE      value
      ---         BLOCKEND  ---      ---       LVL=1
      01000499H   LINE      CODE     ---       #339
      01000499H   LINE      CODE     ---       #340
      01000499H   LINE      CODE     ---       #342
      0100049EH   LINE      CODE     ---       #344
      010004A0H   LINE      CODE     ---       #345
      010004A0H   LINE      CODE     ---       #346
      ---         BLOCKEND  ---      ---       LVL=0

      0100006EH   BLOCK     CODE     ---       LVL=0
      0100006EH   BLOCK     CODE     NEAR LAB  LVL=1
      02000000H   SYMBOL    PDATA    BYTE      del_val_high
      02000001H   SYMBOL    PDATA    BYTE      del_val_low
      02000002H   SYMBOL    PDATA    DWORD     time_out
      ---         BLOCKEND  ---      ---       LVL=1
      0100006EH   LINE      CODE     ---       #351
      0100006EH   LINE      CODE     ---       #352
      0100006EH   LINE      CODE     ---       #355
      01000071H   LINE      CODE     ---       #356
      01000074H   LINE      CODE     ---       #359
      01000076H   LINE      CODE     ---       #363
      01000078H   LINE      CODE     ---       #364
      0100007AH   LINE      CODE     ---       #365
      0100007CH   LINE      CODE     ---       #366
      0100007EH   LINE      CODE     ---       #367
      01000080H   LINE      CODE     ---       #368
      01000082H   LINE      CODE     ---       #369
      01000084H   LINE      CODE     ---       #370
      01000086H   LINE      CODE     ---       #371
      01000088H   LINE      CODE     ---       #372
      0100008AH   LINE      CODE     ---       #373
      01000091H   LINE      CODE     ---       #376
      01000093H   LINE      CODE     ---       #377
      01000095H   LINE      CODE     ---       #378
      01000097H   LINE      CODE     ---       #379
      01000099H   LINE      CODE     ---       #380
      0100009BH   LINE      CODE     ---       #381
      0100009DH   LINE      CODE     ---       #382
      0100009FH   LINE      CODE     ---       #383
LX51 LINKER/LOCATER V3.58                                                             02/22/2012  09:49:47  PAGE 17


      010000A1H   LINE      CODE     ---       #384
      010000A3H   LINE      CODE     ---       #385
      010000A5H   LINE      CODE     ---       #386
      010000ACH   LINE      CODE     ---       #388
      010000AFH   LINE      CODE     ---       #389
      010000B1H   LINE      CODE     ---       #392
      010000B7H   LINE      CODE     ---       #393
      010000B7H   LINE      CODE     ---       #394
      010000BAH   LINE      CODE     ---       #395
      010000BAH   LINE      CODE     ---       #396
      010000BDH   LINE      CODE     ---       #397
      010000BFH   LINE      CODE     ---       #398
      010000C1H   LINE      CODE     ---       #399
      010000C3H   LINE      CODE     ---       #400
      010000C5H   LINE      CODE     ---       #401
      010000C7H   LINE      CODE     ---       #402
      010000C9H   LINE      CODE     ---       #403
      010000CBH   LINE      CODE     ---       #404
      010000CDH   LINE      CODE     ---       #405
      010000CFH   LINE      CODE     ---       #406
      010000D1H   LINE      CODE     ---       #407
      010000D8H   LINE      CODE     ---       #408
      010000D8H   LINE      CODE     ---       #409
      010000D8H   LINE      CODE     ---       #410
      010000D8H   LINE      CODE     ---       #411
      010000D8H   LINE      CODE     ---       #412
      010000D8H   LINE      CODE     ---       #413
      010000D8H   LINE      CODE     ---       #414
      010000D8H   LINE      CODE     ---       #415
      010000D8H   LINE      CODE     ---       #416
      010000D8H   LINE      CODE     ---       #417
      010000D8H   LINE      CODE     ---       #418
      010000DBH   LINE      CODE     ---       #419
      010000DBH   LINE      CODE     ---       #421
      010000DDH   LINE      CODE     ---       #422
      010000DFH   LINE      CODE     ---       #423
      010000E1H   LINE      CODE     ---       #424
      010000E3H   LINE      CODE     ---       #425
      010000E5H   LINE      CODE     ---       #426
      010000E7H   LINE      CODE     ---       #427
      010000E9H   LINE      CODE     ---       #428
      010000EBH   LINE      CODE     ---       #429
      010000EDH   LINE      CODE     ---       #430
      010000EFH   LINE      CODE     ---       #431
      010000F1H   LINE      CODE     ---       #432
      010000F8H   LINE      CODE     ---       #433
      010000FBH   LINE      CODE     ---       #434
      01000102H   LINE      CODE     ---       #435
      01000105H   LINE      CODE     ---       #436
      01000105H   LINE      CODE     ---       #437
      01000105H   LINE      CODE     ---       #440
      01000108H   LINE      CODE     ---       #441
      01000108H   LINE      CODE     ---       #443
      0100010AH   LINE      CODE     ---       #444
      0100010DH   LINE      CODE     ---       #445
      01000110H   LINE      CODE     ---       #446
      01000113H   LINE      CODE     ---       #450
      01000116H   LINE      CODE     ---       #454
      0100011DH   LINE      CODE     ---       #455
      01000126H   LINE      CODE     ---       #456
      01000140H   LINE      CODE     ---       #457
      01000140H   LINE      CODE     ---       #458
      01000160H   LINE      CODE     ---       #459
      01000163H   LINE      CODE     ---       #460
      01000163H   LINE      CODE     ---       #461
LX51 LINKER/LOCATER V3.58                                                             02/22/2012  09:49:47  PAGE 18


      01000165H   LINE      CODE     ---       #462
      01000168H   LINE      CODE     ---       #463
      01000171H   LINE      CODE     ---       #464
      01000178H   LINE      CODE     ---       #465
      0100017AH   LINE      CODE     ---       #466
      0100017AH   LINE      CODE     ---       #467
      0100017CH   LINE      CODE     ---       #470
      0100017EH   LINE      CODE     ---       #483
      0100017EH   LINE      CODE     ---       #485
      01000181H   LINE      CODE     ---       #486
      01000181H   LINE      CODE     ---       #488
      01000183H   LINE      CODE     ---       #489
      01000185H   LINE      CODE     ---       #490
      01000187H   LINE      CODE     ---       #491
      01000189H   LINE      CODE     ---       #492
      0100018BH   LINE      CODE     ---       #493
      0100018DH   LINE      CODE     ---       #494
      0100018FH   LINE      CODE     ---       #495
      01000191H   LINE      CODE     ---       #496
      01000193H   LINE      CODE     ---       #497
      01000195H   LINE      CODE     ---       #498
      0100019CH   LINE      CODE     ---       #499
      0100019CH   LINE      CODE     ---       #500
      0100019CH   LINE      CODE     ---       #501
      0100019CH   LINE      CODE     ---       #502
      0100019CH   LINE      CODE     ---       #503
      0100019CH   LINE      CODE     ---       #504
      0100019CH   LINE      CODE     ---       #505
      0100019CH   LINE      CODE     ---       #506
      0100019CH   LINE      CODE     ---       #507
      0100019CH   LINE      CODE     ---       #508
      0100019CH   LINE      CODE     ---       #509
      0100019FH   LINE      CODE     ---       #510
      010001A1H   LINE      CODE     ---       #511
      010001A3H   LINE      CODE     ---       #512
      010001A5H   LINE      CODE     ---       #513
      010001A7H   LINE      CODE     ---       #514
      010001A9H   LINE      CODE     ---       #515
      010001ABH   LINE      CODE     ---       #516
      010001ADH   LINE      CODE     ---       #517
      010001AFH   LINE      CODE     ---       #518
      010001B1H   LINE      CODE     ---       #519
      010001B3H   LINE      CODE     ---       #520
      010001B6H   LINE      CODE     ---       #521
      010001B6H   LINE      CODE     ---       #522
      010001B6H   LINE      CODE     ---       #523
      010001B6H   LINE      CODE     ---       #524
      010001B6H   LINE      CODE     ---       #525
      010001B6H   LINE      CODE     ---       #526
      010001B6H   LINE      CODE     ---       #527
      010001B6H   LINE      CODE     ---       #528
      010001B6H   LINE      CODE     ---       #529
      010001B6H   LINE      CODE     ---       #530
      010001B6H   LINE      CODE     ---       #531
      010001B9H   LINE      CODE     ---       #532
      010001B9H   LINE      CODE     ---       #535
      ---         BLOCKEND  ---      ---       LVL=0

      ---         MODULE    ---      ---       ?C_INIT
      01000203H   PUBLIC    CODE     ---       ?C_START

      ---         MODULE    ---      ---       ?C?CLDPTR
      01000248H   PUBLIC    CODE     ---       ?C?CLDPTR

      ---         MODULE    ---      ---       ?C?CSTOPTR
LX51 LINKER/LOCATER V3.58                                                             02/22/2012  09:49:47  PAGE 19


      01000261H   PUBLIC    CODE     ---       ?C?CSTOPTR

      ---         MODULE    ---      ---       ?C?ULCMP
      01000283H   PUBLIC    CODE     ---       ?C?ULCMP

      ---         MODULE    ---      ---       ?C?LSTPDATA
      01000294H   PUBLIC    CODE     ---       ?C?LSTPDATA

      ---         MODULE    ---      ---       ?C?LSTKPDATA
      010002A0H   PUBLIC    CODE     ---       ?C?LSTKPDATA



*** WARNING L16: UNCALLED FUNCTION, IGNORED FOR OVERLAY PROCESS
    NAME:    RTC2_INIT/MAIN

*** WARNING L16: UNCALLED FUNCTION, IGNORED FOR OVERLAY PROCESS
    NAME:    RTC0_INIT/MAIN

*** WARNING L16: UNCALLED FUNCTION, IGNORED FOR OVERLAY PROCESS
    NAME:    RTC2_ON/MAIN

*** WARNING L16: UNCALLED FUNCTION, IGNORED FOR OVERLAY PROCESS
    NAME:    RTC2_OFF/MAIN

*** WARNING L16: UNCALLED FUNCTION, IGNORED FOR OVERLAY PROCESS
    NAME:    ADC_INIT/MAIN

*** WARNING L16: UNCALLED FUNCTION, IGNORED FOR OVERLAY PROCESS
    NAME:    ADC_START/MAIN

*** WARNING L16: UNCALLED FUNCTION, IGNORED FOR OVERLAY PROCESS
    NAME:    GET_ADC_VALUE/MAIN

Program Size: data=30.0 xdata=21 const=0 code=1192
LX51 RUN COMPLETE.  7 WARNING(S),  0 ERROR(S)
